:100000000C943A000C9444000C9444000C9444006A
:100010000C9444000C9444000C9444000C94440050
:100020000C9444000C9444000C9444000C94440040
:100030000C9444000C9444000C9444000C94440030
:100040000C9444000C9444000C9444000C94440020
:100050000C9444000C9444000C9444000C94440010
:100060000C9444000C9444000C9444000C94440000
:100070000C94440011241FBECFEFD2E0DEBFCDBFF1
:100080000E9446000C946F000C9400000F931F9385
:100090000E946E003C9A4498509A589A00E111E0F0
:1000A00088B1802788B98BB181278BB982E390E032
:1000B0000E945B00F5CF20E837E004C0F9013197DA
:1000C000F1F701970097D1F7089532E004C0232F8C
:1000D0002A95F1F701970097D1F708950895F894BC
:0200E000FFCF50
:00000001FF
